S00F0000746563626F6F742E7372656325
S3150800000000000120990400086D0400086F04000828
S315080000107104000873040008750400080000000055
S31508000020000000000000000000000000770400083F
S3150800003079040008000000007B0400087D0400081D
S31508000040E9040008E9040008E9040008E9040008CE
S31508000050E9040008E9040008E9040008E9040008BE
S31508000060E9040008E9040008E9040008E9040008AE
S31508000070E9040008E9040008E9040008E90400089E
S31508000080E9040008E9040008E9040008E90400088E
S31508000090E9040008E9040008E9040008E90400087E
S315080000A0E9040008E9040008E9040008E90400086E
S315080000B0E90400080000000000000000E904000848
S315080000C0E90400080000000000000000E904000838
S315080000D000000000E9040008E90400080000000028
S315080000E0E9040008E9040008000000000000000018
S315080000F000000000000000000000000000000000F2
S31508000100000000000000000000000000E9040008EC
S315080001100000000000000000E9040008E9040008E7
S31508000120E9040008E9040008E9040008E9040008ED
S31508000130E9040008000000000000000000000000BC
S31508000140E9040008E9040008E9040008E9040008CD
S31508000150E9040008E9040008E9040008E9040008BD
S31508000160E9040008E9040008E904000800000000A2
S31508000170E9040008E9040008000000000000000087
S31108000180E9040008E9040008E904000886
S3150800018C10B5054C237833B9044B13B10448AFF3B7
S3150800019C00800123237010BD3000002000000000F1
S315080001ACB025000808B5034B1BB103490348AFF348
S315080001BC008008BD0000000034000020B0250008AF
S315080001CC08B501F093FF08BD08B501F09DFF08BD01
S315080001DC08B500F03BF8012008BD08B5642000F00E
S315080001EC05F808BD08B500F007F808BD014B1880DE
S315080001FC704700BF4C00002008B501F025FF0F4BD7
S3150800020C1B68984210D30E4B1B7873B90C4B012202
S3150800021C1A700C4B4FF480429A6101F015FF0A4B89
S3150800022C1B880344054A136008BD054B00221A7047
S3150800023C044B4FF480429A62EFE700BF500000204F
S3150800024C4E000020000800484C000020024B4FF4DA
S3150800025C80429A62704700BF0008004800B597B004
S3150800026C4422002105A802F095F900230093019376
S3150800027C0293039304934FF4007000F0D3FE20BB53
S3150800028C012305934FF4A023069302230F9303220D
S3150800029C109204221192102212920722139214938E
S315080002AC159305A800F0A0FF88B90F230093032324
S315080002BC019300230293039304930421684601F0E7
S315080002CCD3FA30B917B05DF804FB72B6FEE772B60E
S315080002DCFEE772B6FEE7000000B589B000F040F9FB
S315080002ECFFF7BCFF00240394049405940694079422
S315080002FC304BDA6C42F00402DA64DA6C02F004026F
S3150800030C0092009ADA6C42F00102DA64DA6C02F0B6
S3150800031C01020192019ADA6C42F00202DA64DB6C91
S3150800032C03F002030293029B234D22464FF48041AD
S3150800033C284600F069FE4FF4804303930123049387
S3150800034C0594069403A9284600F090FD4FF4004640
S3150800035C03960494059403A9284600F087FD039692
S3150800036C0494059403A94FF0904000F07FFD1823E0
S3150800037C03930494059403A9104800F077FD1048DC
S3150800038C104B0360102343608460C4604FF4403301
S3150800039C03614461047644768476C476047744779C
S315080003AC00F0FAF820B9FFF70BFFFFF70DFFFCE793
S315080003BC72B6FEE700100240000800480004004828
S315080003CC540000200064004082B00A4B1A6E42F0BA
S315080003DC01021A661A6E02F001020092009A9A6DD0
S315080003EC42F080529A659B6D03F080530193019BF2
S315080003FC02B070470010024000B589B00023039381
S3150800040C04930593069307930268144B9A4202D0F9
S3150800041C09B05DF804FB03F5D6339A6D42F0007209
S3150800042C9A659A6D02F000720192019ADA6C42F0A2
S3150800043C0102DA64DB6C03F001030293029B4FF4AE
S3150800044CC0530393022304930323069309230793A8
S3150800045C03A94FF0904000F009FDD9E7006400406D
S3150800046CFEE7FEE7FEE7FEE7FEE7704770477047D4
S3150800047C08B500F085F808BD034AD2F8883043F46D
S3150800048C7003C2F88830704700ED00E0DFF834D00E
S3150800049CFFF7F2FF0C480D490D4A002302E0D45829
S315080004ACC4500433C4188C42F9D30A4A0A4C0023A4
S315080004BC01E013600432A242FBD302F047F8FFF7BF
S315080004CC0BFFFEE700000120000000203000002092
S315080004DC6426000830000020E0040020FEE7704780
S315080004EC10B50A4B4FF0FF329A63DA6300249C630B
S315080004FCDC631A641C649A629C62DA62DC621A63B4
S3150800050C1C63FFF7ECFF204610BD00BF001002402D
S3150800051C104B1B780BB90120704710B504464FF4E5
S3150800052C7A70B0FBF3F30C4A1068B0FBF3F000F0EA
S3150800053CE7FA68B90F2C01D901200AE000222146F6
S3150800054C4FF0FF3000F0A6FA044B1C60002000E0C8
S3150800055C012010BD04000020000000200800002027
S3150800056C10B5032000F084FA0F20FFF7D1FF10B165
S3150800057C0124204610BD0446FFF726FFF9E70000C4
S3150800058C034A1168034B1B780B441360704700BF72
S3150800059C7C00002004000020002800F08A8038B572
S315080005AC044690F82030D3B12268136843F001034F
S315080005BC136001F051FD054623685A6812F0010FC5
S315080005CC10D101F049FD401B0A28F5D9636A43F49A
S315080005DC00336362052384F82030012038BDFFF709
S315080005EC0BFFE1E71A6822F002021A6001F034FDEB
S315080005FC054623685A6812F0020F0DD001F02CFD3F
S3150800060C401B0A28F5D9636A43F400336362052351
S3150800061C84F820300120E1E7227E012A1A680CBFF3
S3150800062C42F0800222F080021A60637E012B226857
S3150800063C13680CBF43F0400323F040031360A37EFA
S3150800064C012B226813680CBF43F0200323F0200308
S3150800065C1360E37E012B226813680CBF23F010038A
S3150800066C43F010031360237F012B226813680CBF19
S3150800067C43F0080323F008031360637F012B2268F9
S3150800068C13680CBF43F0040323F0040313602168BA
S3150800069CA368E268134322691343626913436268C9
S315080006AC013A1343CB6100206062012384F82030A1
S315080006BC94E70120704790F82030013BDBB2012B00
S315080006CC05D9436A43F4802343620120704730B44A
S315080006DC0368D3F8002242F00102C3F800224A69E3
S315080006EC02F01F02012000FA02F2D3F81C026FEA8C
S315080006FC020C20EA0200C3F81C02C869B0B9D3F888
S3150800070C0C020CEA0000C3F80C0248698C88CD6808
S3150800071C44EA0544483043F8304048690C888D68EB
S3150800072C44EA0544483003EBC0004460C869012814
S3150800073C1BD0886980BBD3F804020CEA0000C3F806
S3150800074C0402086970BBD3F814020CEA0000C3F85B
S3150800075C1402096A01292BD0D3F8002222F00102CF
S3150800076CC3F80022002030BC7047D3F80C021043A3
S3150800077CC3F80C0248698C880D6844EA054448306D
S3150800078C43F8304048698C898D6844EA05444830FA
S3150800079C03EBC0004460CCE7D3F804021043C3F85B
S315080007AC0402CEE7D3F814021043C3F81402D0E7B8
S315080007BCD3F81C120A43C3F81C22CDE770B50446BD
S315080007CC90F82050EDB2012D06D0436A43F400236D
S315080007DC43620125284670BD022380F82030026842
S315080007EC136823F00103136001F036FC06462368F0
S315080007FC5B6813F0010F0CD001F02EFC831B0A2B3F
S3150800080CF5D9636A43F400336362052384F8203010
S3150800081CE0E700256562DDE770B590F820C004684E
S3150800082CA4680CF1FF3C5FFA8CFCBCF1010F64D890
S3150800083C14F0E05F5BD0C4F3016C012404FA0CF4E9
S3150800084C1C608B68002B3BD104680D68CB6843EAA7
S3150800085C45550CF118031B01E55003680C690CF19E
S3150800086C180E03EB0E135C600B7D012B35D001685B
S3150800087CD47993791B0443EA046314792343547992
S3150800088C43EA042301EB0C11C1F88C310168D478C6
S3150800089C93781B0443EA046314782343527843EA97
S315080008AC022301EB0C11C1F88831036803EB0C1C0D
S315080008BCDCF8803143F00103CCF88031002021E0CC
S315080008CC04684D68CE68334343EAC5030CF1180E29
S315080008DC4FEA0E1E44F80E30BFE7036803EB0C1301
S315080008ECD3F8841141F48071C3F88411BFE7436AC5
S315080008FC43F400134362012004E0436A43F4802363
S3150800090C4362012070BD90F82030013BDBB2012B0D
S3150800091C01D90020704703689B6803EA8163B3EB2F
S3150800092C816F14BF01200020704790F820C00CF18D
S3150800093CFF3C5FFA8CFCBCF1010F00F2928030B4DC
S3150800094C59B90468E46814F0030F11D1436A43F4E7
S3150800095C00134362012030BC70470468246914F004
S3150800096C030F05D1436A43F4001343620120F2E7EF
S3150800097C01F11B04240105682C5904F00404946045
S3150800098C002C5FD101F11B04240105682C59640D58
S3150800099C1460046801F11B0C4FEA0C1C54F80C404B
S315080009AC04F00204D46004686444646804F00F0418
S315080009BC1461046864446468C4F307249461046885
S315080009CC64446468240C5461026802EB0112D2F880
S315080009DCB8211A70026802EB0112D2F8B821120A71
S315080009EC5A70026802EB0112D2F8B821120C9A70EE
S315080009FC026802EB0112D2F8B821120EDA700268FC
S31508000A0C02EB0112D2F8BC211A71026802EB011230
S31508000A1CD2F8BC21120A5A71026802EB0112D2F8FA
S31508000A2CBC21120C9A71026802EB0112D2F8BC2195
S31508000A3C120EDA7171B90268D36843F02003D360D9
S31508000A4C002088E701F11B04240105682C59E408E9
S31508000A5C54609EE70268136943F020031361002073
S31508000A6C79E7436A43F48023436201207047000008
S31508000A7C0749CA68030203F4E06322F4E06212042D
S31508000A8C120C134343F0BF6343F40033CB60704737
S31508000A9C00ED00E000B5184BDB68C3F30223C3F185
S31508000AAC070CBCF1040F28BF4FF0040C03F1040E1D
S31508000ABCBEF1060F8CBF033B00234FF0FF3E0EFA28
S31508000ACC0CFC21EA0C0199400EFA03F322EA030204
S31508000ADC1143002809DB0901C9B200F1604000F591
S31508000AEC614080F800135DF804FB00F00F00090163
S31508000AFCC9B2024B1954F6E700ED00E014ED00E01C
S31508000B0C0138B0F1807F0BD24FF0E0235861054ACB
S31508000B1CF02182F823100020986107221A61704789
S31508000B2C0120704700ED00E010B40B460A4C6269D0
S31508000B3C42F480226261EFF3108472B601F5807C70
S31508000B4C411A1A685A5004336345FAD184F310884B
S31508000B5C5DF8044B704700BF00200240074B5B69E9
S31508000B6C002B01DB00207047044B054A9A6002F102
S31508000B7C88329A605869C00F704700BF002002403F
S31508000B8C23016745034A536943F000435361002028
S31508000B9C704700BF0020024070B5044601F05CFAAD
S31508000BAC0646144D2B6913F4803F09D0B4F1FF3F68
S31508000BBCF8D001F051FA801BA042F3D3032015E0BC
S31508000BCC0C4B1B690C4A134009D10A4B1B6913F0D1
S31508000BDC010F0CD0074B01221A61002006E00749C9
S31508000BEC4A681A434A60034A1361012070BD002003
S31508000BFCFCE700BF00200240FAC302000C000020EC
S31508000C0C2DE9F04116462B4A1278012A4FD0044694
S31508000C1C0D469846274B01221A704CF25030FFF7B6
S31508000C2CBBFF0746D0B9234B00225A60224B1B68E0
S31508000C3C13F4806F18D0204A136823F4806313606A
S31508000C4C1C4B02221A779CB1631E012B26D94CF237
S31508000C5C5030FFF7A1FF074600F054F8154B002259
S31508000C6C1A703846BDE8F081124B00221A77EAE76B
S31508000C7C114A536943F0010353612E60BFF36F8F1A
S31508000C8CC5F8048001244CF25030FFF785FF07465F
S31508000C9C094A536923EA04035361DDE731462846BA
S31508000CACFFF742FF022CD2D14FF48024EBE7022740
S31508000CBCD7E700BF0C0000200020024010F0010FFF
S31508000CCC04D0054A536943F004035361024A536935
S31508000CDC43F480335361704700200240084B5A692D
S31508000CECC00000F4FF6022F47E72104358615A6902
S31508000CFC42F002025A615A6942F480325A617047CC
S31508000D0C00200240174B1A7FD3B202F0FD02012ACB
S31508000D1C07D0023BDBB2012B15D9124B00221A77EE
S31508000D2C7047114A116821F400711160116841F479
S31508000D3C00611160116821F400611160116841F4B9
S31508000D4C00711160E5E7084B1A6842F480521A6084
S31508000D5C1A6822F480521A601A6842F480621A6081
S31508000D6CDBE700BF0C000020002002402DE9F84309
S31508000D7C3C4B1B78012B71D004460F46394B01228C
S31508000D8C1A704CF25030FFF707FF814600285FD1E6
S31508000D9C344B00225A60344B1B6813F4007F34D052
S31508000DAC314B1B6813F4806F2BD02F4A136823F42E
S31508000DBC806313602B4B03221A772368012B36D0DA
S31508000DCC4FF0FF333B60A568E3682B449D423DD248
S31508000DDC4CF25038244E61682846FFF77FFF404690
S31508000DECFFF7DAFE736923F47E7323F0020373614B
S31508000DFC814650BB0135A368E2681344AB42EAD876
S31508000E0C24E0184B01221A77D7E7174B1B6813F403
S31508000E1C806F08D0144A136823F480631360114B4F
S31508000E2C02221A77C9E70F4B00221A77C5E76068C2
S31508000E3CFFF744FF4CF25030FFF7AEFE81460A4AE4
S31508000E4C536923F00403536100E03D60FFF75AFF32
S31508000E5C044B00221A704846BDE8F8834FF0020985
S31508000E6CF9E700BF0C000020002002400B68002B9D
S31508000E7C00F0C3802DE9F04F83B04FF0000C6246AA
S31508000E8C01254FF0030E4FF00F085C4C48E08368C1
S31508000E9C0EFA0CFA23EA0A0ACB6803FA0CF343EAAD
S31508000EAC0A038360436823EA070A4B68C3F30017EF
S31508000EBC974047EA0A0747603DE0002707FA0BF711
S31508000ECC47EA0A079F60A3686FEA09074E6816F493
S31508000EDC801F0CBF3B4049EA0303A360E3684E68D6
S31508000EEC16F4001F0CBF3B4049EA0303E360636832
S31508000EFC4E6816F4003F0CBF3B4049EA0303636097
S31508000F0C23684E6816F4803F0CBF1F4049EA030756
S31508000F1C276001320B680CF1020C33FA02F669D021
S31508000F2C05FA02F717EA0309F3D04B6803F0030333
S31508000F3C013B012BABD94B6803F00303032B20D0E1
S31508000F4CC3680EFA0CF723EA07078B6803FA0CF347
S31508000F5C3B43C3604B6803F00303022B11D1D7083C
S31508000F6C00EB87073B6A02F0070B4FEA8B0B08FA74
S31508000F7C0BFA23EA0A0A0B6903FA0BF343EA0A0388
S31508000F8C3B6203680EFA0CF723EA07074B6803F073
S31508000F9C030303FA0CF33B4303604B6813F4403F1B
S31508000FACB7D0174E336E43F001033366336E03F036
S31508000FBC01030193019B22F0030303F1804303F51C
S31508000FCC80339F6802F0030B4FEA8B0B08FA0BFA77
S31508000FDC27EA0A0AB0F1904F3FF46FAF094EB042B8
S31508000FEC06D006F58066B0420CBF0227072765E7D0
S31508000FFC2F4663E703B0BDE8F08F70470004014045
S3150800100C00100240000400480AB1816170478162F1
S3150800101C70470000024B186800F4C060704700BFA8
S3150800102C00700040B0F5007F0FD0204B1B6803F40E
S3150800103CC063B3F5806F36D01C4A136823F4C063BB
S3150800104C43F48063136000207047184B1B6803F445
S3150800105CC063B3F5007F24D0144A136823F4C06325
S3150800106C43F400731360124B1B68322101FB03F324
S3150800107C1049A1FB03139B0C0133526912F4806FC0
S3150800108C07D00A49013B4A6912F4806F01D0002B3C
S3150800109CF8D1064B5B6913F4806F0CBF0020032054
S315080010AC7047002070470020704700BF0070004052
S315080010BC0000002083DE1B4330B583B004461E4B6C
S315080010CC9B6D13F0805F0CD0FFF7A4FFB0F5007F83
S315080010DC18D0802C1FD82DD0702C14BF00240124B6
S315080010EC1AE0154DAB6D43F08053AB65AB6D03F051
S315080010FC80530193019BFFF78DFFAB6D23F0805353
S3150800110CAB65E3E7802C04D9A02C8CBF0224012400
S3150800111C02E0002400E0032408490B6823F00703C7
S3150800112C23430B60086800F00700001B18BF01205A
S3150800113C03B030BD0224EFE7001002400020024045
S3150800114C254A9368D26813F00C030ED00C2B06D0E4
S3150800115C042B3FD0082B214818BF0020704702F0FB
S3150800116C0302012A01D0002012E01B4A126812F071
S3150800117C080F194A07BFD2F89420C2F30322126843
S3150800118CC2F30312164951F8220023B30C2B1FD1B4
S3150800119C114BDB6803F00303022B17D00F4A032B02
S315080011AC08BF10460C49CA68CB68C3F3062300FB74
S315080011BC03F3C868C2F302120132B3FBF2F3C0F3AD
S315080011CC416001304000B3FBF0F070470548E9E791
S315080011DC002070470348704700100240005A62020C
S315080011ECE02500080024F400002800F024832DE9EB
S315080011FCF04383B00446984B9D6805F00C05DE68F1
S3150800120C06F00306036813F0100F5FD0F5B10C2D2A
S3150800121C1AD0A369002B00F0BA808F4A136843F0E2
S3150800122C0103136000F018FF0746DFF82C82D8F884
S3150800123C003013F0020F40F0978000F00DFFC01B32
S3150800124C0228F4D9032001E3012EE2D1824B1B6854
S3150800125C13F0020F03D0A369002B00F0EE82206A6C
S3150800126C7D4B1B6813F0080F7B4B12BF1B68D3F81A
S3150800127C94301B0903F0F003984256D8764B1A683B
S3150800128C42F008021A601A6822F0F002216A0A4330
S3150800129C1A605A68E16922F47F4242EA01225A60CE
S315080012AC002D5AD0FFF74CFF6B4B9B68C3F3031307
S315080012BC6A4AD35C03F01F03D840694B1860694B24
S315080012CC1868FFF725F9002840F0C082236813F048
S315080012DC010F7DD0082D72D00C2D6ED06368B3F536
S315080012EC803F00F09480B3F5A02F00F096805A4BFF
S315080012FC1A6822F480321A601A6822F480221A605C
S3150800130C6368002B00F0968000F0A6FE0746DFF80F
S3150800131C4881D8F8003013F4003F59D100F09CFEF0
S3150800132CC01B6428F5D9032090E2FFF7C5FE0028F8
S3150800133C40F08582484B1A6842F008021A601A680F
S3150800134C22F0F002216A0A431A605A68E16922F40B
S3150800135C7F4242EA01225A60A4E7206AFFF7ACFEF4
S3150800136C00289FD0012071E23B4B1A6842F0080214
S3150800137C1A601A6822F0F002216A0A431A605A683F
S3150800138CE16922F47F4242EA01225A609EE7324A18
S3150800139C136823F00103136000F05EFE0746DFF8BE
S315080013ACB880D8F8003013F0020F8FD000F054FE36
S315080013BCC01B0228F5D9032048E2032E8ED1264BF2
S315080013CC1B6813F4003F03D06368002B00F03982C6
S315080013DC236813F0020F5AD0042D47D00C2D43D096
S315080013ECE368002B79D01C4A136843F480731360A6
S315080013FC00F032FE0646184F3B6813F4806F63D133
S3150800140C00F02AFE801B0228F6D903201EE2124A97
S3150800141C136843F48033136072E703F18043A3F532
S3150800142C3C331A6842F480221A601A6842F48032F5
S3150800143C1A6065E700F010FE0746DFF81C80D8F83E
S3150800144C003013F4003FC3D000F006FEC01B64281E
S3150800145CF5D90320FAE100BF00100240C8250008A0
S3150800146C0000002008000020022EB9D1A64B1B68EC
S3150800147C13F4806F03D0E368002B00F0E481A24AD2
S3150800148C5368216923F0F85343EA016353602368D0
S3150800149C13F0080F4CD063699BB39B4AD2F894306F
S315080014AC43F00103C2F8943000F0D6FD0646964F79
S315080014BCD7F8943013F0020F3AD100F0CDFD801B0B
S315080014CC0228F5D90320C1E18F4A5368216923F014
S315080014DCF85343EA01635360D9E78B4A136823F43C
S315080014EC8073136000F0B8FD0646874F3B6813F40B
S315080014FC806FCCD000F0B0FD801B0228F6D90320F3
S3150800150CA4E1814AD2F8943023F00103C2F894304E
S3150800151C00F0A2FD06467C4FD7F8943013F0020F64
S3150800152C06D000F099FD801B0228F5D903208DE121
S3150800153C236813F0040F7ED0734B9B6D13F0805FFA
S3150800154C37D1714B9A6D42F080529A659B6D03F0B8
S3150800155C80530193019B01266C4B1B6813F4807F07
S3150800156C29D0A368012B3CD0052B42D0664BD3F867
S3150800157C902022F00102C3F89020D3F8902022F094
S3150800158C0402C3F89020A368002B40D000F064FD39
S3150800159C0746DFF8748141F28839D8F8903013F091
S315080015AC020F47D100F058FDC01B4845F5D903205A
S315080015BC4CE10026D0E7554A136843F48073136050
S315080015CC00F04AFD0746DFF84481D8F8003013F4DA
S315080015DC807FC6D100F040FDC01B0228F5D9032038
S315080015EC34E1494AD2F8903043F00103C2F89030FE
S315080015FCC9E7454BD3F8902042F00402C3F8902073
S3150800160CD3F8902042F00102C3F89020BBE700F013
S3150800161C23FD0746DFF8F08041F28839D8F8903078
S3150800162C13F0020F06D000F017FDC01B4845F5D97C
S3150800163C03200BE1E6B9236813F0200F35D0636A53
S3150800164CE3B1314AD2F8983043F00103C2F8983026
S3150800165C00F002FD06462C4FD7F8983013F0020F0F
S3150800166C23D100F0F9FC801B0228F5D90320EDE004
S3150800167C254A936D23F080539365DCE7224AD2F80A
S3150800168C983023F00103C2F8983000F0E5FC0646C2
S3150800169C1D4FD7F8983013F0020F06D000F0DCFC7B
S315080016AC801B0228F5D90320D0E0A36A002B00F092
S315080016BCCC80022B17D00C2D00F0CD80124A136863
S315080016CC23F08073136000F0C7FC04460E4D2B689C
S315080016DC13F0007F00F0A88000F0BEFC001B022867
S315080016ECF5D90320B2E0084BDB6803F00301E26A84
S315080016FC91420DD00C2D00F0AC80034B1B6813F0F7
S3150800170C806F2FD00120A1E000100240007000402D
S3150800171C03F07002216B0139B2EB011FEAD103F415
S3150800172CFE42616BB2EB012FE4D103F07842A16B58
S3150800173CB2EBC16FDED103F4C001E26B5208013A79
S3150800174CB1EB425FD6D103F0C063226C5208013A62
S3150800175CB3EB426FCED1414B1B6813F0007F49D0D7
S3150800176C002073E03D4A136823F08073136000F081
S3150800177C73FC0546394E336813F0007F06D000F02B
S3150800178C6BFC401B0228F6D903205FE0334AD1686C
S3150800179C334B0B40E16A0B43616B43EA0123A16BA4
S315080017AC43EAC163216B013943EA0113E16B49082A
S315080017BC013943EA4153216C4908013943EA41632B
S315080017CCD360136843F080731360D36843F0807357
S315080017DCD36000F041FC0446204D2B6813F0007FC3
S315080017EC06D100F039FC001B0228F6D903202DE09F
S315080017FC00202BE0194B1A6842F080721A60DA68DE
S3150800180C42F08072DA6000F027FC0446134D2B6810
S3150800181C13F0007F06D100F01FFC031B022BF6D930
S3150800182C032013E0002011E00C4AD1680D4B0B4045
S3150800183CD36000200AE001207047012006E0012051
S3150800184C04E0012002E0012000E0002003B0BDE81E
S3150800185CF0830120FAE70120F8E700BF00100240E8
S3150800186C8C809D01FCFFEEFE002876D02DE9F04118
S3150800187C0D4604465E4B1B6803F007038B420AD2DF
S3150800188C5B4A136823F007030B431360136803F0D2
S3150800189C07038B4263D1236813F0020F65D0A16846
S315080018AC544A926802F0F002914240F29C80514AE6
S315080018BC936823F0F0030B439360236813F0010F2E
S315080018CC39D06268032A09D0022A26D062BB494B52
S315080018DC1B6813F0020F06D1012082E0454B1B68EA
S315080018EC13F0007F3DD043498B6823F00303134361
S315080018FC8B6000F0B1FB06463E4F41F28838BB6858
S3150800190C03F00C036268B3EB820F14D000F0A4FB4F
S3150800191C801B4045F3D9032063E0364B1B6813F450
S3150800192C003FE0D101205CE0324B1B6813F4806F5A
S3150800193CD9D1012055E0236813F0020F18D0A268FC
S3150800194C2C4B9B6803F0F0039A4211D229498B68F9
S3150800195C23F0F00313438B600AE001207047012043
S3150800196C3FE001203DE001203BE013F0010FA8D138
S3150800197C1F4B1B6803F00703AB420AD91C4A1368B2
S3150800198C23F007032B431360136803F00703AB42DA
S3150800199CE9D1236813F0040F06D0164A936823F48A
S315080019ACE063E1680B439360236813F0080F07D0D4
S315080019BC104A9368216923F4605343EAC103936080
S315080019CCFFF7BEFB0B4B9B68C3F303130A4AD35CA6
S315080019DC03F01F03D840094B1860094B1868FEF72B
S315080019EC97FDBDE8F08113F0010F7FF46AAFA6E707
S315080019FC0020024000100240C82500080000002004
S31508001A0C08000020054B9B68C3F30223044AD35CE9
S31508001A1C03F01F03034A1068D840704700100240B1
S31508001A2CD82500080000002072B6704762B67047C9
S31508001A3CF0B58BB0FFF7E6FF3D4BA3FB00308009F2
S31508001A4C3C4A02F12405002402E00232AA4266D07E
S31508001A5C92F800E092F801C00EEB0C030133C3EBCD
S31508001A6C431103EB8103B0FBF3F103FB11010029CE
S31508001A7CEBD1B0FBF3F39CB2631E9BB2B3F5806F4C
S31508001A8CE3D22D4D2D4B2B6000262E766E76AE7638
S31508001A9C0127EF762E776E77AE60EE600EF1FF3E7D
S31508001AAC4FEA0E432B610CF1FF3C4FEA0C536B616A
S31508001ABC6C602846FEF770FD4FF09043196903F5E4
S31508001ACC806318691B691E4A1269C0F30010C3F3B8
S31508001ADCC0039B0043EA4003C1F3C0310B43C2F376
S31508001AECC03243EAC203174A13700596069607973F
S31508001AFC5B0143F4C043009301964FF6E0730293DF
S31508001B0C04230393049608970E23099369462846DB
S31508001B1CFEF7D1FD2846FEF751FE0BB0F0BDAA2103
S31508001B2C094800F0A1FA4FF0000CE646A9E700BFF9
S31508001B3CD34D621030260008840000200064004053
S31508001B4C00080048800000201026000830B589B02F
S31508001B5C0246114B1B7843F45073029300230493EB
S31508001B6C0593069101AB02A90C48FEF755FE08B180
S31508001B7C09B030BD00F068FA00F13204074D01993E
S31508001B8C2846FEF7C0FE0028F2D000F024FB00F031
S31508001B9C5BFAA042F3D9EBE7800000208400002012
S31508001BAC30B589B003460D460A4A147801AA0021B5
S31508001BBC0948FEF7BAFE50B944F44074019BA34297
S31508001BCC06D1039B23B9059B2B70012000E000204E
S31508001BDC09B030BD800000208400002008B5FFF74E
S31508001BEC23FF08BD10B500F0F7F900B910BDFEF7D4
S31508001BFCEFFA0028FAD000F0B7FAFEF771FC00F0FD
S31508001C0CFBF900F0EDF920F0604020F07F00044B62
S31508001C1C986000F0E5F94468FFF708FFA047E5E788
S31508001C2C00ED00E082B170B50C46551EADB20D4400
S31508001C3C0135461AA3192246013412781A7000F097
S31508001C4CCAFAAC42F6D170BD704700002DE9F84FC0
S31508001C5C8046FEF783FF164B4FF400421A610025A7
S31508001C6C08F1040BAA46D8F800402C440BEB0503E4
S31508001C7CD3E9006700F0AFFA32463B462146504698
S31508001C8CFEF7BEFF814660B9D4E90023BB4208BF04
S31508001C9CB24208D10835B5F5007FE4D14FF00109F9
S31508001CAC01E04FF00009FEF76DFF4846BDE8F88FD6
S31508001CBC0020024038B50D46104B98421AD00446FF
S31508001CCC0F4B99420DD10D4C2368AB4207D02046D9
S31508001CDC40F8045B4FF400722946FFF7A3FF204631
S31508001CEC38BDFFF7B3FF38B1C5F30803002BEBD0AB
S31508001CFC0024F4E7034CF7E70024F0E7B0020020D1
S31508001D0C00280008AC0000202DE9F84306460C46CE
S31508001D1C91461F4621F4FF7828F001080368B3F1B1
S31508001D2CFF3F0BD03368434510D104343368E41AAB
S31508001D3C34444D4608F500784F4416E040F8048BB9
S31508001D4C4FF400724146FFF76DFFEBE7414630460C
S31508001D5CFFF7B0FF06460028E7D1002015E015F876
S31508001D6C013B04F8013BBD420ED000F034FA331D9A
S31508001D7CE31AB3F5007FF2D341463046FFF79AFFD4
S31508001D8C064620B1041DEAE70120BDE8F8830020C9
S31508001D9CFBE700004FF0FF33024A1360024A136058
S31508001DAC704700BFAC000020B00200200B4601F1C2
S31508001DBCFF3C1049091A8C4515D80F49884214D38B
S31508001DCC411E1944B1F1016F11D210B520F4FF71FF
S31508001DDC21F00101084CA14201460CBF07480848EE
S31508001DECFFF792FF10BD00207047002070470020B7
S31508001DFC704700BFFFFF0F0800280008B00200203C
S31508001E0CAC0000202DE9F04186B04A1E2F4B1B1A58
S31508001E1C9A4251D820F4FF6424F007042C4B9C42B8
S31508001E2C4FD3431E0B44B3F1016F4CD20144091B2B
S31508001E3CC1F3CF25C1F30A0109B10135ADB2FEF7DD
S31508001E4C8DFE244B4FF400421A61002301930123A3
S31508001E5C04935DB3013DADB204F5006303EBC525F0
S31508001E6C1D4EDFF87C801D4F00F0B5F9D6F8E0352D
S31508001E7C99B24FF6FF7291421ABF07EA832303F110
S31508001E8C006343469C4234BF04F17843E31ADB0AE9
S31508001E9C03930123029305A901A8FEF767FF38B936
S31508001EAC04F50064AC42DFD1012402E0012400E011
S31508001EBC0024FEF767FE00E00024204606B0BDE8C5
S31508001ECCF0810024F9E70024F7E700BFFFFF0F08AD
S31508001EDC00280008002002400070FF1F00FCFF03CA
S31508001EEC00000408104B1B68B3F1FF3F19D000B56E
S31508001EFC83B00D4A536891680B44D1680B44116939
S31508001F0C0B4451690B4491690B44D26913445B42E7
S31508001F1C019301AA04210548FFF748FF03B05DF8B1
S31508001F2C04FB0120704700BFB00200208C29000872
S31508001F3C104AD2F80038D2F804180B44D2F808180C
S31508001F4C0B44D2F80C180B44D2F810180B44D2F8E0
S31508001F5C14180B44D2F818180B44D2F88C09D8422A
S31508001F6C05D0054B984214BF00200120704701206C
S31508001F7C704700BF002000082255AAEE08B50C4B86
S31508001F8C1B68B3F1FF3F06D10A4B1B68B3F1FF3F41
S31508001F9C07D1012008BD0648FFF758FE0028F3D1E3
S31508001FACF8E70448FFF752FE003818BF0120F1E79E
S31508001FBCB0020020AC00002000487047002800083A
S31508001FCC08B5FFF7E7FE08BD08B5FFF7EFFE08BD35
S31508001FDC08B5FFF717FF08BD08B5FFF7A9FF08BD39
S31508001FEC08B5FFF7E9FF08BD08B5FFF77BFF00B991
S31508001FFC08BDFFF7C3FFFBE74FF0E02300221A6189
S3150800200C5A619A617047000008B5FFF7F5FF4FF063
S3150800201CE023044A5A6100229A6105211961024B90
S3150800202C1A6008BD7F380100B40400204FF0E02385
S3150800203C1B6913F4803F03D0024A136801331360FB
S3150800204C704700BFB404002008B5FFF7EFFF014B3B
S3150800205C186808BDB404002008B5FFF7E7FF014B64
S3150800206C186808BDB404002008B500F0B4F8FCE7FD
S3150800207C08B500F0A5F8012803D00B4B1B78012BEB
S3150800208C00D008BDFFF7E0FF084B1B68084A12682A
S3150800209C134403F57A739842F3D3034B00221A7050
S315080020ACFFF7A0FDEDE700BFBC040020B804002034
S315080020BCC004002008B5054B1B78012B00D008BDC1
S315080020CCFFF7C2FF024B1860F9E700BFBC040020FB
S315080020DCC004002008B5044B01221A70FFF7EAFF6A
S315080020ECFFF7C6FF08BD00BFBC04002008B5FFF704
S315080020FC75FD00F06CF8FFF787FFFFF761FF00F03E
S3150800210C0DF8FFF7E7FF08BD08B500F064F8FFF710
S3150800211C8DFF00F00FF8FFF7ABFF08BD08B500F010
S3150800212C75F8FFF785FC024B01221A7008BD00BF33
S3150800213C2C00002000B583B00DF107010848FFF705
S3150800214C2FFD012802D003B05DF804FB054B0122D4
S3150800215C1A709DF80710024800F072F8F3E700BFF2
S3150800216CC40400202C0000207047000008B5054B5D
S3150800217C1B78012B02D000F05DF808BDC9B2FFF739
S3150800218CE5FCF8E72C000020054B1B7833B1023B25
S3150800219CDBB2022B34BF00200820704700207047A2
S315080021AC2C000020054B1B7833B1023BDBB2022B0B
S315080021BC34BF002008207047002070472C000020F0
S315080021CC08B500F02FF8003818BF012008BD08B56F
S315080021DCFEF703F808BD08B5FEF704F808BD0000BD
S315080021EC034BFE221A70587002229A81704700BF60
S315080021FCCC040020427883781B0443EA0223027835
S3150800220C1343C07843EA006070470000044B002271
S3150800221C1A721A61DA729A819A725A72704700BFE8
S3150800222CCC040020024B187A003818BF01207047DE
S3150800223CCC040020014B0022DA727047CC04002033
S3150800224C70B50378FF2B40D00446A94A127A012AA6
S3150800225C5FD1C93B352B00F26F81DFE813F0F5002F
S3150800226C6D016D0169016D016D0161010F014D0172
S3150800227C39016D016D016D016D016D016D016D0108
S3150800228C6D016D016D016D016D016D016D016D01C4
S3150800229C6D016D016D016D016D016D016D016D01B4
S315080022AC6D016D016D016D016D016D016D016D01A4
S315080022BC6D01A80073005B0090006D016D016D0146
S315080022CCCA006D01DB00DF00EC00894C0023637249
S315080022DC01252572FF22227010226270A370FFF767
S315080022EC53FFE070FFF75EFF2071FFF75BFF000AF4
S315080022FC6071A571E5710823A381FFF761FE7C4B1C
S3150800230CDB7A012B00F01C81794BB3F90C100029F0
S3150800231C46DC70BDFFF738FF627890420ED9744DD3
S3150800232C2969681CFFF77EFCFF232B7062782B69E2
S3150800233C13442B6163780133AB8129E02220FFF724
S3150800234C4FFFDCE7FFF720FF6378834213D2201D8B
S3150800235CFFF750FF0146664D28616278681CFFF747
S3150800236C61FCFF232B7062782B6913442B6163780D
S3150800237C0133AB810CE02220FFF732FFBFE75C4D3F
S3150800238CFF232B700430FFF735FF28610123AB813F
S3150800239C574BDB7A012B00F0D380554BB3F90C1055
S315080023AC53480123C37289B2FFF7E0FEB1E7504DDB
S315080023BCFF232B700430FFF71DFF2D690646B0B1BD
S315080023CC2E44002415F8013B1C44E4B2FFF703FF26
S315080023DCB542F7D1464B01225A701C7100225A712C
S315080023EC9A71DA719A70DA7008229A81D0E7002409
S315080023FCF0E73F4BFF221A703E4A1A6100225A70C8
S3150800240C9A70DA70072119715A719A71DA71082261
S3150800241C9A81BDE70020FFF7E3FE70E7344BFF22F5
S3150800242C1A7000225A70597A9970DA701A715A71A0
S3150800243C06229A81ACE72E4B00221A725A72FF2298
S3150800244C1A7001229A81A3E7294B1D69FFF79CFE96
S3150800245C621C411E2846FFF7B7FD58B1244CFF23D2
S3150800246C2370FFF791FE0138236903442361012386
S3150800247CA3818DE73120FFF7B3FE40E7FFF784FE13
S3150800248C01386378984212DD194BFF221A70012223
S3150800249C9A81617879B1A21C154B1869FFF794FDDE
S315080024AC90B1134A617813690B44136127E722200C
S315080024BCFFF796FE23E7FFF797FD00287FF41FAF7B
S315080024CC3120FFF78DFE1AE73120FFF789FE16E754
S315080024DC074CFF23237000256570A570FFF754FE83
S315080024ECE07025716571A5710723A38150E700BFBC
S315080024FCCC04002054260008134B1D690430FFF742
S3150800250C79FE01462846FFF763FD28B10E4BFF22DC
S3150800251C1A7001229A813BE73120FFF761FEEEE63D
S3150800252CFFF760FB084BFF221A7001229A812FE7EE
S3150800253C3120FFF755FEE2E62020FFF751FEDEE6D6
S3150800254C1020FFF74DFEDFE6CC04002070B50D4DCC
S3150800255C0D4C641BA4100026A64209D10B4D0C4C3D
S3150800256C00F020F8641BA4100026A64205D170BD05
S3150800257C55F8043B98470136EEE755F8043B98475F
S3150800258C0136F2E75C2600085C2600085C26000883
S3150800259C6026000802440346934200D1704703F8AC
S315080025AC011BF9E7F8B500BFF8BC08BC9E46704796
S311080025BCF8B500BFF8BC08BC9E46704786
S315080025C800000000000000000102030406070809CD
S315080025D80000000001020304A0860100400D030064
S315080025E8801A060000350C0040420F0080841E0041
S315080025F800093D0000127A000024F40000366E0136
S315080026080048E801006CDC022E2E2F6F70656E629A
S315080026186C742F41524D434D345F53544D33324CED
S31508002628342F63616E2E630005020602060307034C
S315080026380803090309040A040B040C040C050D0510
S315080026480E050F050F061006100710084F70656E61
S30908002658424C54008E
S3090800265CB1010008B2
S309080026608D010008D2
S3150800266400093D0001000000100000000000000001
S315080026740000000000000000000000000100000047
S315080026840000000000000000000000000400000034
S7050800049955
